S02700002E2E5C62696E5C64656D6F70726F675F6F6C696D6578696E6F5F73746D33322E7372656308
S3150800600000500020C16900080F6A0008116A0008DC
S31508006010136A0008156A0008176A000800000000DD
S31508006020000000000000000000000000196A0008D7
S315080060301B6A0008000000001D6A0008D56A0008EF
S31508006040236A0008256A0008276A0008296A0008E2
S315080060502B6A00082D6A00082F6A0008316A0008B2
S31508006060336A0008356A0008376A0008396A000882
S315080060703B6A00083D6A00083F6A0008416A000852
S31508006080436A0008456A0008476A0008496A000822
S315080060904B6A00084D6A00084F6A0008516A0008F2
S315080060A0536A0008556A0008576A0008596A0008C2
S315080060B05B6A00085D6A00085F6A0008616A000892
S315080060C0636A0008656A0008676A0008696A000862
S315080060D06B6A00086D6A00086F6A0008716A000832
S315080060E0736A0008756A0008776A0008EE11AA55EF
S315080060F010B5054C237833B9044B13B10448AFF3F4
S3150800610000800123237010BD6C00002000000000F1
S31508006110B06B0008084B10B51BB108490848AFF327
S3150800612000800848036803B910BD074B002BFBD055
S31508006130BDE81040184700BF0000000070000020AE
S31508006140B06B00086C00002000000000154B002B07
S3150800615008BF134B9D46A3F5803A00218B460F4690
S315080061601348144A121A00F0F7FC0F4B002B00D004
S3150800617098470E4B002B00D09847002000210400BA
S315080061800D000D48002802D00C48AFF3008000F03F
S31508006190BDFC2000290000F009FC00F0A3FC00BFAC
S315080061A00000080000500020000000000000000069
S315080061B06C00002094000020000000000000000091
S315080061C0F0B5002421E0134D15F8147005EB4405CD
S315080061D095F801E007EB0E0505FB000548F6A04C0F
S315080061E09CFBF5F605FB16C66EB99CFBF5F5ADB23C
S315080061F00D80013DADB2B5F5806F04D2177083F8F6
S3150800620000E00120F0BD0134E4B2112CDBD90020F6
S31508006210F0BD00BF846B000830B58BB0012108467D
S3150800622000F00CFB0121082000F008FB4FF48073F6
S31508006230ADF8243048238DF82730344C09A9204678
S3150800624000F070FA4FF40073ADF8243018238DF877
S31508006250273003238DF8263009A9204600F062FA74
S3150800626001214FF4EA1000F0AFFA01214FF0007057
S3150800627000F0F2FA264D284600F0C6F806A800F007
S31508006280E1F901AB0DF105020DF106014FF4FA70C3
S31508006290FFF796FF00248DF81E408DF81F408DF8F5
S315080062A020408DF821408DF822408DF823408DF846
S315080062B01A408DF81B409DF80530013B8DF81C30BF
S315080062C09DF80430013B8DF81D30BDF80630ADF859
S315080062D0183006A9284600F0B3F88DF812408DF854
S315080062E0134001238DF81430ADF80840ADF80A4084
S315080062F0ADF80C40ADF80E40ADF810408DF81530ED
S3150800630002A800F025F90BB030BD00BF000C014013
S315080063100064004008B5FFF77FFF08BDBFF34F8F45
S315080063200449CA6802F4E062034B1343CB60BFF327
S315080063304F8FFEE700ED00E00400FA0500B587B0D0
S3150800634000210D4800F0E0F990B101AA00210A48A1
S3150800635000F088F940F26763019A9A4208D19DF8DD
S315080063600F30FF2B04D19DF810300BB9FFF7D6FF7D
S3150800637007B05DF804FB00BF0064004008B5FFF7EE
S31508006380DDFF08BD30B583B00121042000F056FAC0
S3150800639003238DF8063010238DF80730202502A92F
S315080063A021F8045D044C204600F0BCF92946204635
S315080063B000F008FA03B030BD0008014010B500F03F
S315080063C083FB0E4B1B68C31AB3F5FA7F14D3044636
S315080063D00B4B1B783BB90122094B1A70202109483F
S315080063E000F0EEF906E00022054B1A702021054858
S315080063F000F0E8F9014B1C6010BD00BF88000020C2
S315080064008C0000200008014008B50C4B98420AD1C0
S3150800641001214FF0007000F02DFA00214FF00070B6
S3150800642000F028FA08BD01214FF0806000F022FA3A
S3150800643000214FF0806000F01DFA08BD006400409E
S31508006440036823F002030360036843F00103036053
S31508006450002300E00133426812F0010F03D14FF622
S31508006460FF729342F6D1436813F0010F6BD08B7914
S31508006470012B04D1036843F08003036003E003683B
S3150800648023F080030360CB79012B04D1036843F022
S315080064904003036003E0036823F0400303600B7ABC
S315080064A0012B04D1036843F02003036003E003686B
S315080064B023F0200303604B7A012B04D1036843F0D1
S315080064C01003036003E0036823F0100303608B7A6C
S315080064D0012B04D1036843F00803036003E0036853
S315080064E023F008030360CB7A012B04D1036843F039
S315080064F00403036003E0036823F0040303608A7857
S31508006500CB781B0643EA82730A7943EA02434A793F
S3150800651043EA02530A88013A1343C361036823F026
S3150800652001030360002300E00133426812F0010F03
S3150800653003D04FF6FF729342F6D1436813F0010F6A
S3150800654003D000207047002070470120704700BF25
S3150800655070B4837A012202FA03F3394AD2F8001298
S3150800656041F00101C2F80012D2F81C12DC432140A6
S31508006570C2F81C12027BB2B9314AD2F80C12214079
S31508006580C2F80C12817AC688458845EA064548311C
S3150800659042F83150857A8688018841EA06414835AD
S315080065A002EBC5025160027B012A16D1244AD2F8B1
S315080065B00C121943C2F80C12817A0688458845EAF6
S315080065C00645483142F83150857A8688C18841EABD
S315080065D00641483502EBC5025160C27A32B91849FC
S315080065E0D1F804222240C1F8042205E01449D1F862
S315080065F004221A43C1F8042202892AB91049D1F89B
S3150800660014221440C1F814420289012A05D10C4902
S31508006610D1F814221A43C1F81422427B012A05D163
S315080066200749D1F81C221343C1F81C32044AD2F890
S31508006630003223F00103C2F8003270BC704700BF75
S315080066400064004000238371C3710372437283722E
S31508006650C3728370C370032303710223437101233A
S315080066600380704710B401F11B031B01C35803F0E4
S315080066700403DBB2137233B901F11B031B01C358C0
S315080066805B0D136005E001F11B031B01C358DB0812
S31508006690536001F11B031B01C418C35803F002031E
S315080066A05372636803F00F03937263681B0AD3740B
S315080066B000EB0113D3F8B841D472D3F8B841240AD1
S315080066C01473D3F8B841240C5473D3F8B841240E84
S315080066D09473D3F8BC41D473D3F8BC41240A147418
S315080066E0D3F8BC41240C5474D3F8BC311B0E9374F4
S315080066F021B9C36843F02003C36003E0036943F08C
S315080067002003036110BC704719B9C06800F0030084
S315080067107047012903D1006900F003007047002083
S31508006720704700BFF0B4CB7803F00F02154613F09C
S31508006730100F01D08D7815430B78E3B10668002356
S3150800674016E001229A400C8832EA04040FD19C0014
S315080067500F27A74026EA070605FA04F42643CC784D
S31508006760282C01D1426102E0482C00D10261013394
S31508006770072BE6D906600B88FF2B1ED9466800232F
S3150800678018E003F108040122A2400C8832EA040446
S315080067900FD19C000F27A74026EA070605FA04F43E
S315080067A02643CC78282C00D14261CC78482C00D1DD
S315080067B002610133072BE4D94660F0BC704700BF7D
S315080067C0016170474161704730B4002802DA1A4BFC
S315080067D0DB6901E0184B5B68C0F3034582B200F43D
S315080067E04014B4F5401F07D123F07063124D6C684E
S315080067F024F070646C6011E010F4801F06D0032446
S31508006800AC4023EA040343F0706307E0440D240117
S3150800681002FA04F423EA040343F0706319B1410D44
S3150800682009018A401343002802DA034AD36101E0CA
S31508006830014A536030BC70470000014021B1054B46
S315080068409A69104398617047024A936923EA0000DF
S31508006850906170470010024021B1054BDA69104378
S31508006860D8617047024AD36923EA0000D0617047AD
S315080068700010024021B1054B1A6910431861704790
S31508006880024A136923EA00001061704700100240AB
S3150800689082B00023019300932C4A136843F4803393
S315080068A013602A4B1B6803F400330093019B0133E2
S315080068B00193009B1BB9019BB3F5A06FF1D1234B44
S315080068C01B6813F4003F02D00123009301E0002364
S315080068D00093009B012B36D11D4B1A6842F010021B
S315080068E01A601A6822F003021A601A6842F0020255
S315080068F01A60A3F580535A685A605A685A605A68EB
S3150800690042F480625A605A6822F47C125A605A68C5
S3150800691042F4E8125A601A6842F080721A600B4B09
S315080069201B6813F0007FFAD0084B5A6822F003025E
S315080069305A605A6842F002025A60044B5B6803F0D8
S315080069400C03082BF9D102B0704700BF00100240B3
S315080069500020024008B5FFF79BFF08BD08B50E4B9F
S315080069601A6842F001021A6059680C4A0A405A60CD
S315080069701A6822F0847222F480321A601A6822F4A5
S3150800698080221A605A6822F4FE025A604FF41F02E7
S315080069909A60FFF7DFFF08BD001002400000FFF80D
S315080069A008B5FFF7EFFC00F071F808BD08B5FFF76A
S315080069B0F7FFFFF7AFFCFFF701FDFFF7DFFCFAE78C
S315080069C007498D460749084A084B9A42BEBF51F8FF
S315080069D0040B42F8040BF8E70548804705480047CA
S315080069E000500020BC6B0008000000206C0000204E
S315080069F05D6900084D6100081F49204A002301E02F
S31508006A0041F8043B9142FBD3FFF7D0FFFEE7FEE7D0
S31508006A10FEE7FEE7FEE7FEE7FEE7FEE7FEE7FEE740
S31508006A20FEE7FEE7FEE7FEE7FEE7FEE7FEE7FEE730
S31508006A30FEE7FEE7FEE7FEE7FEE7FEE7FEE7FEE720
S31508006A40FEE7FEE7FEE7FEE7FEE7FEE7FEE7FEE710
S31508006A50FEE7FEE7FEE7FEE7FEE7FEE7FEE7FEE700
S31508006A60FEE7FEE7FEE7FEE7FEE7FEE7FEE7FEE7F0
S31508006A70FEE7FEE7FEE7FEE76C0000209400002034
S31508006A80014B1860704700BF9000002008B50A4BFC
S31508006A901B680A4AA2FB03239B09013B084A536069
S31508006AA0F021084B83F82310002090600723136019
S31508006AB0FFF7E6FF08BD00BF00000020D34D6210B7
S31508006AC010E000E000ED00E0014B1868704700BFD9
S31508006AD090000020024A136801331360704700BF14
S31508006AE09000002008B5074B044613B10021AFF308
S31508006AF00080054B1868836A03B19847204600F062
S31508006B0033F800BF00000000AC6B00080E4B70B5F0
S31508006B101E460E4C0025E41AA410A54204D056F8C9
S31508006B20253098470135F8E700F020F8084B094C5E
S31508006B301E46E41AA4100025A54204D056F82530AE
S31508006B4098470135F8E770BD64000020640000200E
S31508006B50640000206800002003460244934202D0E5
S31508006B6003F8011BFAE77047FEE70000F8B500BF17
S31508006B70F8BC08BC9E467047F8B500BFF8BC08BC10
S31508006B809E46704705020602060307030803090323
S31508006B9009040A040B040C040C050D050E050F0563
S31508006BA00F06100610071008430000000400002016
S30908006BB000000000D3
S30D08006BB498F5FF7F01000000BF
S31508006BBC00A24A04000000000000000000000000CB
S31508006BCC00000000000000000000000000000000AB
S31508006BDC00000000A86B0008000000000000000080
S31508006BEC000000000000000000000000000000008B
S31508006BFC000000000000000000000000000000007B
S31508006C0C000000000000000000000000000000006A
S31108006C1C0000000015610008F160000887
S7050800600092
